:103E3D000FC30FBF0FBB0FB60FB20FAC0FA70FA164
:103E4D000F9B0F950F8E0F870F800F780F700F68D8
:103E5D000F5F0F550F4B0F410F360F2B0F1F0F120B
:103E6D000F060EF80EEA0EDB0ECC0EBC0EAB0E9A44
:103E7D000E880E750E620E4E0E390E240E0E0DF7B7
:103E8D000DDF0DC70DAE0D940D790D5E0D410D2499
:103E9D000D070CE80CC90CA90C890C680C460C23F9
:103EAD000C000BDC0BB80B930B6E0B480B210AFAB5
:103EBD000AD30AAC0A840A5B0A330A0A09E109B774
:103ECD00098E0965093B091108E808BE0895086CBB
:103EDD000842081907F107C807A0077807500729F6
:103EED00070206DB06B5068F066A0645062105FDA7
:103EFD0005DA05B70595057405530532051204F36A
:103F0D0004D404B60498047B045F04430428040D10
:103F1D0003F303DA03C103A90391037A0363034D8A
:103F2D0003370322030E02F902E602D302C002AEEA
:103F3D00029C028B027A026A025A024B023C022D4B
:103F4D00021F0211020301F601E901DD01D001C5D5
:103F5D0001B901AE01A30198018E0184017A0171AD
:103F6D000168015F0156014D0145013D0135012EED
:103F7D000126011F01180111010B010400FE00F8BB
:103F8D0000F200EC00E600E100DC00D600D100CC30
:103F9D0000C800C300BE00BA00B600010C01010448
:103FAD0002011E030A96040132050404060064078B
:103FBD00010108000009015A0E01010F0001120054
:103FCD006413010114013C1501FA1664FA17FFFF81
:103FDD001D00072000072400022701012F013C309E
:103FED0002023201033500023603073CFFFF3DFF9D
:103FFD00FF180002191E461A00021B00022D32C8BE
:10400D002E0001FAFAFA18000019FFFF1A00001B22
:10401D0000002D32C82E0001FAFAFA18000019FF1F
:10402D00FF1A00001B00002DFFFF2EFFFFFAFAFA0A
:10004800900786E0FEA3E0FF7457BE0010D39F40E0
:100058000C903FA712001EE493F599804C90001471
:10006800E0D394044014900786E0FEA3E0FF903F9D
:10007800A712001EE493F599802F900014E0D39402
:10008800034014900786E0FEA3E0FF903FBC1200F7
:100098001EE493F5998012900786E0FEA3E0FF9096
:1000A8003FD112001EE493F59990078612000E9036
:1000B8000786E0FEA3E0FF746C6F4E7003751300B3
:1000C80022900072E0B402087401900072F0D20C21
:1000D80090013AE090002AF090013BE090002BF06C
:1000E80090013CE090002CF0A20AB3401690013A2F
:1000F800E0700C90013BE0700690013CE0600280EB
:1001080002C20A90013AE0B4300F90013BE0B447D4
:100118000890013CE0643B60028004D20B8002C27C
:100128000BE558B40102800302024B900057E0F53A
:1001380067900062E0F569900063E0F56A900074EA
:10014800E0F56B90007AE0900029F090007CE0F5F3
:100158006690007DE0F568900080E0F5659000818C
:10016800E0F564900090E0900041F0900091E090FC
:100178000042F0900092E0900043F0900093E090ED
:100188000044F0900094E0900045F0900095E090D5
:100198000046F0900096E0900047F0900097E090BD
:1001A8000048F0900099E0900033F090009AE090B9
:1001B8000034F090009BE0900035F090009CE090B7
:1001C8000036F0900079E0B4011790000A740FF03F
:1001D800A374FFF090000CE4F0A3F074029000798F
:1001E800F0900079E0B4035990000CE0FEA3E0FF22
:1001F80090000AE0FCA3E0FD120003741012419D78
:10020800740812418FEF900026F0EF700674FF908B
:100218000026F07400900079F090000BE090002721
:10022800F090000AE0900028F0900026E0900789FE
:10023800F0900027E090078AF0900028E090078B64
:10024800F0803F900081E07006755801756400A247
:100258000AB3402E90013AE090002AF090013BE06A
:1002680090002BF090013CE090002CF090002AE0E8
:10027800700C90002BE0700690002CE06002800269
:10028800C20AE5677003756702E56970037569025C
:100298007E877FA4E5678E048F05FF12417F8C3926
:1002A8008D3AE56A75F0FAA4FFAEF0E5698E048F21
:1002B80005FF12417F8C3D8D3E90004FE0F5619027
:1002C800004DE0FE900069E0B5061890004CE0FE95
:1002D800900068E0B5060C90004BE0FE900059E0F5
:1002E8006E606F900069E07006900068E0600674C8
:1002F80000900059F0900069E0B402089000497439
:1003080001F08005900049E4F0900068E0B402082C
:1003180090004A7401F0800590004AE4F09000686B
:10032800E0600690004AE060028005756103800382
:10033800756104E559B55802D20C900068E0900048
:100348004CF0900069E090004DF0900059E090006A
:100358004BF0740190009EF0740190009FF07400BF
:100368009000A0F074009000A1F074009000A2F03A
:1003780074009000A3F074009000A4F07401900041
:10038800A5F074019000A6F074009000A7F0740026
:100398009000A8F074009000A9F074009000AAF0F2
:1003A80074009000ABF074019000ACF07401900000
:1003B800ADF074009000AEF074009000AFF07400DF
:1003C8009000B0F074009000B1F074009000B2F0AA
:1003D8007401900362F07401900363F07400900359
:1003E80064F07401900365F07400900366F0740083
:1003F800900367F07400900368F074009003A2F013
:1004080074019003A3F074009003A4F074019003A6
:10041800A5F074009003A6F074009003A7F0740090
:100428009003A8F074009003E2F074009003E3F0E6
:1004380074009003E4F074019003E5F074009003F5
:10044800E6F074009003E7F074009003E8F074019C
:10045800900422F07400900423F07401900424F0B6
:100468007401900425F07400900426F07400900440
:1004780027F07400900428F022E5B554F7F5B5E5A7
:10048800B554FDF5B5C2A2D297C2A1C292C207E582
:10049800B554FBF5B5755104E55104F55290004F7C
:1004A800E0F561900025E4F0C209E5B554FEF5B524
:1004B800C28E758D00758B00754C007526007525EC
:1004C80000D28E22750A00750900AE09AF0A74576A
:1004D800BE00039F5003020589903FA712001EE447
:1004E8009390004E1241B50FBF00010EE0FC903F03
:1004F800A712001EECFEE493FFEEC39F5026AE0940
:10050800AF0A0FBF00010E903FA712001EAE09AF41
:100518000AE493FC903FA712001EE49390004E1249
:1005280041B5ECF0AE09AF0A903FA712001EE49364
:1005380090004E1241B5E0FC903FA912001EECFC61
:10054800E493FDECD39D4019903FA912001EE4935B
:10055800FC903FA712001EE49390004E1241B5ECA8
:10056800F0AE09AF0A74022FFF50010E8E098F0AF0
:10057800780A740126F6500418E436F6400302049B
:10058800D222750A00750900AE09AF0A7415BE00BB
:10059800039F5003020657903FFE12001EE49390FB
:1005A800004E1241B50FBF00010EE0FC903FFE1255
:1005B800001EECFEE493FFEEC39F5026AE09AF0A7F
:1005C8000FBF00010E903FFE12001EAE09AF0AE4F5
:1005D80093FC903FFE12001EE49390004E1241B52A
:1005E800ECF0AE09AF0A903FFE12001EE4939000B3
:1005F8004E1241B5E0FC90400012001EECFCE49362
:10060800FDECD39D401990400012001EE493FC902D
:100618003FFE12001EE49390004E1241B5ECF0AE7E
:1006280009AF0A740F6F4E7006750A15750900AE8A
:1006380009AF0A74022FFF50010E8E098F0A780A3B
:10064800740126F6500418E436F640030205902299
:10065800750A00750900AE09AF0A7415BE00039F3C
:10066800500302072590401312001EE49390004E99
:100678001241B50FBF00010EE0FC90401312001E9E
:10068800ECFEE493FFEEC39F5026AE09AF0A0FBFFE
:1006980000010E90401312001EAE09AF0AE493FC4D
:1006A80090401312001EE49390004E1241B5ECF0F6
:1006B800AE09AF0A90401312001EE49390004E1248
:1006C80041B5E0FC90401512001EECFCE493FDECF3
:1006D800D39D401990401512001EE493FC904013DE
:1006E80012001EE49390004E1241B5ECF0AE09AF33
:1006F8000A740F6F4E7006750A15750900AE09AFBA
:100708000A74022FFF50010E8E098F0A780A7401AD
:1007180026F6500418E436F6400302065E22750AEF
:1007280000750900AE09AF0A7415BE00039F500397
:100738000207F390402812001EE49390004E1241E5
:10074800B50FBF00010EE0FC90402812001EECFE21
:10075800E493FFEEC39F5026AE09AF0A0FBF000116
:100768000E90402812001EAE09AF0AE493FC904098
:100778002812001EE49390004E1241B5ECF0AE0929
:10078800AF0A90402812001EE49390004E1241B523
:10079800E0FC90402A12001EECFCE493FDECD39D93
:1007A800401990402A12001EE493FC904028120041
:1007B8001EE49390004E1241B5ECF0AE09AF0A74F6
:1007C8000F6F4E7006750A15750900AE09AF0A74E9
:1007D800022FFF50010E8E098F0A780A740126F63F
:1007E800500418E436F6400302072C22054D220572
:1007F8004C22054EC2CF2290F800E49364066002B2
:1008080080FE75840175A70075FF80900788E4F065
:1008180075C91075A70F75A1C775A70075D900759B
:10082800CEFF75A70F75F1FE75F2FF75F33775F4F6
:100838007C75A4BA75A5FF75A60775AE0075AFFFE0
:1008480075D48175D5FF75D6FF75D7FFC296C29549
:10085800C2A0C20DC297E5B554BFF5B5E5B554DFE2
:10086800F5B5E5B554EFF5B5E5B5547FF5B5E5B59E
:1008780054F7F5B5E5B554FDF5B575A70075A201B2
:1008880075A14775F80975BC0175BE0475BD6C7511
:10089800BE0775BDA075BE0875BD0175BC0075BBEA
:1008A8001875BC2075BA0875E88075D11375A70F3F
:1008B80075E10575E20075C74075970075978074F6
:1008C8000A12416F7597C0E5975420700280F87539
:1008D8008F0275A700D2AF75980075A90C75A70F80
:1008E80075AB4375ADFB75AC1E75A70075891175A1
:1008F8008E00758C00758A00D2A9D28C758D007512
:100908008B00D2ABD28E75CD0075CC0075CA007540
:10091800CB00D2ADC2CFD2CA75910475920075933F
:10092800CD75EF0675D94075CF01900786E4F0A321
:10093800F0751300751400C299D20AC20E12048110
:1009480074C8F51875170012276C75A70FE5FB908A
:10095800001AF0E5FA90001BF0E5F990001CF0751C
:10096800A70090F800E493F5081228A3122DDD9053
:100978000789E0900026F090078AE0900027F09021
:10098800078BE0900028F090078CE0900029F09009
:10099800078DE0F56790078EE0F56990078FE0F521
:1009A8006A900790E0F56B900791E0F566900792E2
:1009B800E0F568900793E0F565900794E0F564909A
:1009C8000795E090002AF0900796E090002BF090B1
:1009D8000797E090002CF0900798E0900041F09085
:1009E8000799E0900042F090079AE0900043F09059
:1009F800079BE0900044F090079CE0900045F09041
:100A0800079DE0900046F090079EE0900047F09028
:100A1800079FE0900048F09007A0E0900033F09026
:100A280007A1E0900034F09007A2E0900035F09024
:100A380007A3E0900036F07400900082F090013A2D
:100A4800E0700C90013BE0700690013CE060028091
:100A580004C20A8002D20A90F807E493900021F0B9
:100A6800900021E0440A900021F0900021E054FE1B
:100A7800900021F07406900012F07402900013F0B8
:100A880090F802E493900014F07403900015F07449
:100A980003900016F07429900017F0740590001860
:100AA800F0900014E0B404067404900018F090006C
:100AB80014E0B403067403900018F074059000194C
:100AC800F090F804E49390001DF0740090001EF07C
:100AD80090F805E49390001FF090F806E4939000D6
:100AE80020F074FF900022F07453900125F0747583
:100AF800900126F07462900127F07461900128F04B
:100B08007472900129F0747590012AF07420900194
:100B18002BF0743490012CF0744590012DF0744141
:100B280090012EF0745490012FF07420900130F051
:100B38007434900131F07453900132F07450900184
:100B480033F090007AE0D394014006740090007A64
:100B5800F0755801755901740390004CF01200C9E2
:100B68001204CC900014E0B40405120658801190C9
:100B78000014E0D39404400512058A800312072666
:100B8800122798E5B554FEF5B5900025E4F09007D6
:100B980086E4F0A3F0752400752300754800752AD3
:100BA80000752900754900753200753100754A00D5
:100BB800755400755500755A0075510475520175C4
:100BC800343C7533007571007570007572CD7556BB
:100BD800007557007543007544007545007546005B
:100BE800755B00754700754200754100900006E48A
:100BF800F0A3F0900008E4F0A3F0755F00756000C2
:100C080090000E74FDF0A374E8F0900023E4F074F3
:100C180064900024F0C200D201C202D203754D00D4
:100C2800756E00C294C293C287C290C291C20C7EF4
:100C3800017F00900028E012419D900027E02FFFDF
:100C480050010E90000AEEF0A3EFF0900026E0703D
:100C58000674FF900026F090000AE0FEA3E0FFEF84
:100C6800D394FFEE940F400790000AE4F0A3F074C9
:100C780000900071F07400900079F0740090008288
:100C8800F0740090008DF074009000B4F0E5687086
:100C980003756804743A90074EF074FD90074FF09E
:100CA8009003D4E0900414F0D2B0D2B7D2A7D2A661
:100CB800D2B1D2A3C207A2B6B39204A2B3B392052B
:100CC800D29CD2EC75CF01A298B34005C2981231DC
:100CD80041E5136006A299B3B340028005C2991298
:100CE80036B1E51464016005E514B4040280D5E565
:100CF8004DD39405400CE55AC394C85002055A7563
:100D08004D00E572C394F0501A787012003FAE702F
:100D1800AF71EFD394E8EE94034008057275710043
:100D2800757000C28E7E047F00E54C12419DE58DF2
:100D380075F004A4FDACF0EF2DFDEE3CFCE58B75E1
:100D4800F04084FF7E00ED2FFFEC3EFE8E258F26BF
:100D5800D28EA2B6300401B35003020E9FA2B63061
:100D68000401B35003020E9FA2B640670554A20EB9
:100D7800400575FFA0D20EE5B54401F5B5900024F5
:100D8800E4F0E554D3956740487C877DA4AE25AF51
:100D98002612403D8E238F24E5482FFF50010E7404
:100DA8000112418F8E238F24852448755401C28EE9
:100DB800758D00758B00754C00D28E7403BE0003D0
:100DC8009F50069000257401F0E543B4060375436F
:100DD80000D204A2B6B35003020E9FC20490006B67
:100DE800E060181237F2A200B34008E5B54408F5F0
:100DF800B58006E5B554F7F5B58002C20090006EDF
:100E0800E06018123947A202B34008E5B54402F57C
:100E1800B58006E5B554FDF5B58006E5B554FDF594
:100E2800B5A207B34004D2878002C287900059E078
:100E38006004D2908002C29090004AE0B40104D2CB
:100E4800948002C294900049E0B40104D2938002D5
:100E5800C293A209B34004D2918002C291900018B3
:100E6800E0FE900014E0C39E4009900014E0D39483
:100E780008400974FB900023F012048190001DE0E3
:100E8800601590001DE0FE900017E06E600974FE8A
:100E9800900023F0120481C2CA7E017F00E54E1241
:100EA800419DE5CD2FFF50010E8E278F28D2CAE530
:100EB80066B4014890000EE0FCA3E0FDEFC39DEE90
:100EC8009C4039B208E52A45296013A208B34008B6
:100ED800E5B54404F5B58006E5B554FBF5B59000D5
:100EE8000EE0FEA3E0FF900010E0FCA3E0FDEF2D74
:100EF800FDEE3CFC90000EECF0A3EDF0A2B3300543
:100F080001B35003020FEDA2B3300501B350030241
:100F18000FEDA2B35003020FE60555A20E4005756A
:100F2800FFA0D20EE5B54401F5B5900024E4F0E544
:100F380055D395695003020FE47CEA7D60AE27AF74
:100F48002812403D8E298F2AE56A12419D74FF8E32
:100F5800048F05FF12417F8C298D2AE5492DFD500C
:100F6800010C74018C068D0712418F8E298F2A85FA
:100F78002A49A209B34015746412419D900067E0A4
:100F88008E048F05FF12417F8C298D2A755501909B
:100F9800000EE0FEA3E0FFAC27AD2812000390008E
:100FA8000EEEF0A3EFF0E568FF12417F740AFF121E
:100FB800417F90007BE08C068D0712419D74148E52
:100FC800048F05FF12417F900010ECF0A3EDF0C2F2
:100FD800CA75CD0075CC00754E00D2CAD205A2B331
:100FE800B34002C205900025E0B40107E556C3945A
:100FF8000640030215FEE56E90274BF828287390EB
:101008000059E0C39402400302115BE551D39401F7
:10101800500302115BE55175F040A4FFAEF0900358
:101028001212001EE0C395455018E55175F040A412
:10103800FFAEF090031112001EE0F52E752D000290
:10104800115BE55175F040A4FFAEF090031012005B
:101058001EE0C3954540030210F7E55175F040A422
:10106800FFAEF090031112001EE55175F040A4FF89
:10107800AEF0E0FC90030F12001EECFEE0FFEEC3A2
:101088009FFEE5518E0475F040A4FFAEF09003106A
:1010980012001EE0F40425458C0088F0A4FFAEF091
:1010A800E5518F048E0575F040A4FFAEF090031251
:1010B80012001EE55175F040A4FFAEF0E0FA90036F
:1010C8001012001EEAFEE0FFEEC39FFECDCCCD8ECF
:1010D8000712417FE55175F040A4FFAEF090030F71
:1010E80012001EE02DFD50010C8C2D8D2E8064E524
:1010F8005175F040A4FFAEF090030F12001EE551A9
:1011080075F040A4FFAEF0E0FC90030E12001EEC58
:10111800FEE0FFEEC39F8545F0A4FFAEF0E5518FDA
:10112800048E0575F040A4FFAEF090031012001E67
:10113800E0FECDCCCD8E0712417FE55175F040A47D
:10114800FFAEF090030E12001EE02DFD50010C8C36
:101158002D8D2E756E010215FE900059E0C3940284
:10116800400302130E90004FE0D395515003021232
:10117800B7E55175F040A4FFAEF090031812001EB9
:10118800E0C395455018E55175F040A4FFAEF090C6
:10119800031712001EE0F52C752B000212B7E5515B
:1011A80075F040A4FFAEF090031612001EE0C39540
:1011B800454003021253E55175F040A4FFAEF0908C
:1011C800031712001EE55175F040A4FFAEF0E0FCD5
:1011D80090031512001EECFEE0FFEEC39FFEE551E2
:1011E8008E0475F040A4FFAEF090031612001EE0C6
:1011F800F40425458C0088F0A4FFAEF0E5518F0477
:101208008E0575F040A4FFAEF090031812001EE59D
:101218005175F040A4FFAEF0E0FA90031612001EDC
:10122800EAFEE0FFEEC39FFECDCCCD8E0712417FD4
:10123800E55175F040A4FFAEF090031512001EE0D2
:101248002DFD50010C8C2B8D2C8064E55175F040E0
:10125800A4FFAEF090031512001EE55175F040A4EE
:10126800FFAEF0E0FC90031412001EECFEE0FFEE6F
:10127800C39F8545F0A4FFAEF0E5518F048E057538
:10128800F040A4FFAEF090031612001EE0FECDCC95
:10129800CD8E0712417FE55175F040A4FFAEF09066
:1012A800031412001EE02DFD50010C8C2B8D2CE533
:1012B80051B40122E561D39401401BE551C3955611
:1012C8005014E545C39405500D90035FE0A829B874
:1012D8000006952A40028003755102E551B5612246
:1012E80090004FE0D395514019E55175F040A4FFA7
:1012F800AEF090031712001EE0A823B8000695244C
:10130800400280020561756E020215FE900059E0E8
:10131800B4022AE55175F040A4FFAEF0900317120D
:10132800001EE0F52C752B00E55175F040A4FFAECA
:10133800F090030E12001EE0F52E752D0090005956
:10134800E0B4030F900051E0F52C752B00752E00CA
:10135800752D00756E030215FEE55175F040A4FF6A
:10136800AEF090032012001EE0C3955A4003021409
:1013780035900049E07036E551D394014029AE23F9
:10138800AF24AC2DAD2EEDD39FEC9E401AE55175E0
:10139800F040A4FFAEF090031E12001EE0A829B88A
:1013A8000005D3952A5002800215518034E551D3A7
:1013B80094024029AE23AF24AC2DAD2EEDD39FEC83
:1013C8009E401AE55175F040A4FFAEF090031E123E
:1013D800001EE0A829B80005D3952A5002800215FE
:1013E80051E551B55236E551C39561502FE551C3CA
:1013F80095565028AE23AF24AC2BAD2CEFD39DEEE1
:101408009C4019E55175F040A4FFAEF090031F12FF
:10141800001EE0A829B80006952A4002800205515E
:10142800C292E55165526005C207755A00756E048F
:101438000215FEE55175F040A4FFAEF090031A12B4
:10144800001EE0B40117E55175F040A4FFAEF0901E
:10145800032012001EE0240AC3955A400302150B0C
:10146800753064752F00A207B3500B900060E0241C
:1014780005C39545400302150BE55175F040A4FFDF
:10148800AEF090031D12001EE0C395454064E5517F
:1014980075F040A4FFAEF090031C12001EE55175D4
:1014A800F040A4FFAEF0E0FC90031B12001EECFE1F
:1014B800E0FFEEC39F8545F0A4FFAEF0E5518F0431
:1014C8008E0575F040A4FFAEF090031D12001EE0DB
:1014D800FECDCCCD8E0712417FE55175F040A4FFBB
:1014E800AEF090031B12001EE02DFD50010C8C2F56
:1014F8008D30AE23AF24AC2FAD30EFD39DEE9C40A2
:1015080002D207756E050215FEE551B40109900077
:1015180059E0C3940240030215DE900358E0D395C6
:101528004550030215DE900356E0C39545504090A0
:101538000357E0FE900355E0F4042EFE900356E0B6
:10154800F40425458E0088F0A4FFAEF0900358E01F
:10155800FC900356E0F4042C8E048F05FF12417FA3
:10156800900355E02DFD50010C8C2B8D2C802C9078
:101578000355E0FE900354E0F4042E8545F0A4FFE3
:10158800AEF0900356E08E048F05FF12417F900362
:1015980054E02DFD50010C8C2B8D2CE551C3956129
:1015A800502FE551C395565028AE23AF24AC2BAD30
:1015B8002CEFD39DEE9C4019E55175F040A4FFAE89
:1015C800F090031F12001EE0A829B80006952A40D3
:1015D800028003755102900049E0B40106E55164A8
:1015E8000160028003755102E55165526005C2072A
:0615F800755A00756E003B
:10274B0002100702116102131402136102143B02FF
:02275B00151156
:1015FE00900050E02402A823B80007D3952440029F
:10160E00C207900025E0B40109900059E0C394038D
:10161E004003021784900049E060030216D4E5519E
:10162E00D394014034E55175F040A4FFAEF0900321
:10163E001412001EE0A823B8001FD39524401AE50B
:10164E005175F040A4FFAEF090031F12001EE0A8EB
:10165E0029B80005D3952A500280021551E551D3C1
:10166E009401402FE55175F040A4FFAEF0900312A7
:10167E0012001EE0C39545501AE55175F040A4FFC7
:10168E00AEF090031E12001EE0A829B80005D395F7
:10169E002A500280021551E551D394014021E551A3
:1016AE00D39556401AE55175F040A4FFAEF0900365
:1016BE001E12001EE0A829B80005D3952A500280FC
:1016CE00021551021779E551D394024034E5517554
:1016DE00F040A4FFAEF090031412001EE0A823B851
:1016EE00001FD39524401AE55175F040A4FFAEF0CB
:1016FE0090031F12001EE0A829B80005D3952A50AA
:10170E000280021551E551D39402402FE55175F038
:10171E0040A4FFAEF090031212001EE0C395455098
:10172E001AE55175F040A4FFAEF090031E12001E94
:10173E00E0A829B80005D3952A500280021551E57C
:10174E0051D394024021E551D39556401AE5517577
:10175E00F040A4FFAEF090031E12001EE0A829B8C0
:10176E000005D3952A500280021551E5516552604D
:10177E0005C207755A00900060E0D3954550099058
:10178E000054E0C395455002C207900059E0700323
:10179E000219E7A2A5B34008A2A4B340030219D0D0
:1017AE00AE35AF367441D39F749C9E40057835128A
:1017BE00003FAE35AF36EFB48806EEB413028003A9
:1017CE000219ADA2A55003021870900059E0B401A1
:1017DE000B90004FE0D3956140020561900059E0F7
:1017EE00B40253E55175F040A4FFAEF09003201201
:1017FE00001EE0C3955A503E90004FE0D3955140E5
:10180E0020E551C395565019E55175F040A4FFAE31
:10181E00F090031412001EE0A823B8000695244091
:10182E00028002055190004FE0F561E5516552606E
:10183E0005C207755A00900059E0B4032590004F79
:10184E00E0D395514007E551C395564002800205FD
:10185E005190004FE0F561E55165526005C2077584
:10186E005A00A2A450030219AD900059E0B4016EC3
:10187E00900049E07035E551D394014029E551754A
:10188E00F040A4FFAEF090031E12001EE0A829B88F
:10189E00000FD3952A400A1551755A008551618063
:1018AE000385516180037561018033E551D3940244
:1018BE004029E55175F040A4FFAEF090031E1200D2
:1018CE001EE0A829B8000FD3952A400A1551755A63
:1018DE00008551618003855161800375610290001E
:1018EE0059E0D3940150030219A1E55175F040A4BB
:1018FE00FFAEF090032012001EE0C3955A40030283
:10190E0019A1900049E07041E551D394014034E5AE
:10191E005175F040A4FFAEF090031112001EE0A826
:10192E0023B8001FD39524401AE55175F040A4FF4B
:10193E00AEF090031E12001EE0A829B80005D39544
:10194E002A500280021551803FE551D39402403453
:10195E00E55175F040A4FFAEF090031112001EE0A9
:10196E00A823B8001FD39524401AE55175F040A462
:10197E00FFAEF090031E12001EE0A829B80005D39A
:10198E00952A500280021551E55165526005C20735
:10199E00755A00E556B40704055F8003755F00E5D0
:1019AE0064B4010EAE35AF36EF64407005EE649C44
:1019BE006002800EA2A54003755801A2A4400375D3
:1019CE005802A2A5B3B35006A2A4B3B34002800638
:1019DE00753600753500021AD5A2A5B34008A2A42B
:1019EE00B34003021AC1AE35AF367441D39F749C17
:1019FE009E4005783512003FAE35AF36EFB48806FF
:101A0E00EEB413028003021AC1A2A5406F900068C3
:101A1E00E0605A90004AE0B4010790004AE4F0807A
:101A2E000690004A7401F090004AE070057561035B
:101A3E00800375610490004AE0B40104D2948002E0
:101A4E00C294E551B4041AE55175F040A4FFAEF00E
:101A5E0090031E12001EE0A829B80005D3952A5047
:101A6E00028008755103C207755A00800375610420
:101A7E00E556B40704055F8003755F00A2A44033EA
:101A8E00900069E06021900049E0B40107900049A0
:101A9E00E4F080069000497401F0900049E0B40132
:101AAE0004D2938002C293E556B40704055F800307
:101ABE00755F00A2A5B3B35006A2A4B3B3400280D3
:101ACE0006753600753500E558655960069000823A
:101ADE00E06003021C5DC29C751400751300C2CA3F
:101AEE00E55890275DF82828738012122DDD800DA1
:0D1AFE00122EB68008122F8F800312306860
:0F275D00021AF7021AF9021AFE021B03021B08E6
:101B0B00900029E090007AF0E567900057F0E569C6
:101B1B00900062F0E56A900063F0E56B900074F062
:101B2B00E56690007CF0E56890007DF0E56590003F
:101B3B0080F0E564900081F090002AE090013AF08B
:101B4B0090002BE090013BF090002CE090013CF0DA
:101B5B00900041E0900090F0900042E0900091F0F6
:101B6B00900043E0900092F0900044E0900093F0DE
:101B7B00900045E0900094F0900046E0900095F0C6
:101B8B00900047E0900096F0900048E0900097F0AE
:101B9B00900033E0900099F0900034E090009AF0C0
:101BAB00900035E090009BF0900036E090009CF0A8
:101BBB007400900082F07453900125F074759001BD
:101BCB0026F07462900127F07461900128F0747212
:101BDB00900129F0747590012AF0742090012BF07C
:101BEB00743490012CF0744590012DF074419001E8
:101BFB002EF0745490012FF07420900130F0743457
:101C0B00900131F07453900132F07450900133F025
:101C1B009003D4E0900414F0743A90074EF074FDE6
:101C2B0090074FF01200C9900004E4F0A3F090006D
:101C3B00067475F0A37430F09000087475F0A374FB
:101C4B0030F0855859D2CA754C00D29C741B900049
:101C5B0023F0E556C394065005E551B55203021C1B
:101C6B00F1C207E55175F040A4FFAEF090032212CC
:101C7B00001EE030E003D38001C39296E55175F06E
:101C8B0040A4FFAEF090032312001EE030E003D31C
:101C9B008001C39295E55175F040A4FFAEF090031F
:101CAB002412001EE030E003D38001C3920DE552F5
:101CBB00B40306E551640260028002D2A0E552B47F
:101CCB000206E551640160028002D2A0855152AE3A
:101CDB0029AF2A7405BE00039F5007E545D3940531
:101CEB0050028002D292E556D394055003021DFB9D
:101CFB00C207E551D394014073E55175F040A4FF41
:101D0B00AEF090031E12001EE0A829B80007D39571
:101D1B002A40021551E5516552604EE55175F04070
:101D2B00A4FFAEF090032212001EE030E003D3803C
:101D3B0001C39296E55175F040A4FFAEF0900323DA
:101D4B0012001EE030E003D38001C39295E551757C
:101D5B00F040A4FFAEF090032412001EE030E0032D
:101D6B00D38001C3920D855152021DFBE556B4067B
:101D7B00279000ACE030E003D38001C39296900033
:101D8B00ADE030E003D38001C392959000AEE0301C
:101D9B00E003D38001C3920DE556B407279000A54D
:101DAB00E030E003D38001C392969000A6E030E0D0
:101DBB0003D38001C392959000A7E030E003D3805A
:101DCB0001C3920DE556B4082790009EE030E00366
:101DDB00D38001C3929690009FE030E003D3800143
:101DEB00C392959000A0E030E003D38001C3920D25
:101DFB00900072E06058E54575F00284FF7E00901C
:101E0B00014E12001EE0F55CE54775F00A84FF7E7B
:101E1B000090024E12001EE0F55EE55C255ED39449
:101E2B0064400BE55C255EC39464F55C8003755CD4
:101E3B0000E55C75F00284FF7E008F5CEFC394338A
:101E4B005007EF24CDF55C8003755CFF801CE545E6
:101E5B0075F00284FF7E0090014E12001EE075F0BB
:101E6B000284FF7E00EF24CDF55CE595C3955C40C5
:101E7B0004C2A28002D2A2A207B34005E556B40762
:101E8B00037572CDE595C395724004C2A18002D251
:101E9B00A1900083E0702BE54575F00284FF7E0076
:101EAB0090018012001EE075F00284FF7E00EF248B
:101EBB00CDF55DE595C3955D4004D2978002C29741
:101ECB008027900083E0B40105A2B2B340028004E6
:101EDB00C2978015900083E0B40206A2B2B3B34060
:101EEB00028004C2978002D297E543C39406400355
:101EFB000224F7A2EDB350030224F7C2EDE54360D1
:101F0B00030220597E017F00E5BE12419DE5BD2FE6
:101F1B00FF50010E900000EEF0A3EFF0900029E0CF
:101F2B00B401177E0F7FFF900000E0FCA3E0FD12D1
:101F3B000003900000EEF0A3EFF0900079E0B40204
:101F4B005B900000E0FEA3E0FF90000AE0FCA3E042
:101F5B00FDEDD39FEC9E400F900000E0F8A3E090C6
:101F6B00000AC8F0A3C8F0900000E0FEA3E0FF90C9
:101F7B00000CE0FCA3E0FDEFD39DEE9C400F900026
:101F8B0000E0F8A3E090000CC8F0A3C8F0900000AC
:101F9B00E0FEA3E0FF740412418F8F44900079E0C0
:101FAB007060900000E0FEA3E0FF90000AE0FCA34D
:101FBB00E0FDEFD39DEE9C400D120003900000EE70
:101FCB00F0A3EFF08007900000E4F0A3F090000086
:101FDB00E0FEA3E0FF741012419D900026E08E04FA
:101FEB008F05FF12417F900000ECF0A3EDF0740021
:101FFB00D39D74019C4008900001E0F5448003756B
:10200B0044FFE54475F00AA4FFAEF074198E048FFB
:10201B0005FF12417F8D45ED2532FFAE3150010E8C
:10202B00740112418F8F45854532753100EFD39482
:10203B00624003754562900072E064016006900097
:10204B0066E060028005754301800375BB17E543AD
:10205B00B4010280030221497E017F00E5BE1241DB
:10206B009DE5BD2FFF50010E900000EEF0A3EFF0A9
:10207B00900072E0B4017EE53445336025AC33AD9E
:10208B00341DBDFF011C8F028E038C068D07903E05
:10209B003D12002EE493FE740193FFEFC39AEE9B67
:1020AB004002800578331241C7AE33AF3474B3BEF0
:1020BB000025D39F4021900000E0FCA3E0FD0FBF63
:1020CB0000010E903E3D12002EE493FE740193FF2F
:1020DB00EDC39FEC9E40028005783312003FAE3378
:1020EB00AF34E56B12419D74648E048F05FF124172
:1020FB007F8D478033900066E0602D900000E0FEFE
:10210B00A3E0FFEFD39400EE9408400F900066E03D
:10211B00B40104C2098002D209800D900066E0B4BC
:10212B000104D2098002C209900072E064026006C9
:10213B00900066E0600575BB168003754302E543AE
:10214B00B4020280030222377E017F00E5BE1241FA
:10215B009DE5BD2FFF50010E900000EEF0A3EFF0B8
:10216B00900072E0B4027EE53445336025AC33ADAC
:10217B00341DBDFF011C8F028E038C068D07903C16
:10218B00D312002EE493FE740193FFEFC39AEE9BE0
:10219B004002800578331241C7AE33AF3474B3BEFF
:1021AB000025D39F4021900000E0FCA3E0FD0FBF72
:1021BB0000010E903CD312002EE493FE740193FFAA
:1021CB00EDC39FEC9E40028005783312003FAE3387
:1021DB00AF34E56B12419D74648E048F05FF124181
:1021EB007F8D478033900066E0602D900000E0FE0D
:1021FB00A3E0FFEFD39400EE9408400F900066E04D
:10220B00B40104C2098002D209800D900066E0B4CB
:10221B000104D2098002C209900072E07003754775
:10222B0000900066E07002C20975BB1FE543B40362
:10223B00457E017F00E5BE12419DE5BD2FFF50019C
:10224B000E900000EEF0A3EFF0740912419D74E6BE
:10225B008E048F05FF12417F8C418D42E54A2DFD87
:10226B0050010C74018C068D0712418F8E418F42E9
:10227B0085424A75BB19E543B4040280030223DF90
:10228B007E017F00E5BE12419DE5BD2FFF50010E83
:10229B00900000EEF0A3EFF0740412418F8F4BE52A
:1022AB0065B40102800302236C756C00756C00E54C
:1022BB006CD394074003022359E56C900041124103
:1022CB00B5E0D3954B501AE56C9000411241B5E047
:1022DB00F404254BFEE56C9000371241B5EEF0800F
:1022EB0017E56C9000411241B5E0C3954BFEE56CD0
:1022FB009000371241B5EEF0E56CC39404400990A1
:10230B000084E0C3956C503BE56C6029E56C900054
:10231B00371241B5FEE0FFEE90003FE0D39F401334
:10232B00E56C9000371241B5E090003FF0E56C9002
:10233B000040F0800E900037E090003FF07400906A
:10234B000040F0786C740126F640030222BA90002C
:10235B0040E0F4042408F556E556D394054002C238
:10236B0092E565D39401402FE54BD3946E4004D294
:10237B000F8002C20F755605E565B40205A20FB3B7
:10238B0040028003755607E565B40306A20FB3B38D
:10239B0040028003755607E55765566008E5510402
:1023AB00F552855657E556B40708E5B54480F5B5A3
:1023BB008006E5B5547FF5B5E55664066005E55630
:1023CB00B40808E5B54410F5B58006E5B554EFF54E
:1023DB00B575BB13E543B4050280030224F37E01FC
:1023EB007F00E5BE12419DE5BD2FFF50010E900011
:1023FB0000EEF0A3EFF0740412418F8F46E564B446
:10240B00020280030224F0756C00756C00E56CD33E
:10241B00940340030224A7E56C9000331241B5E00E
:10242B00D39546501AE56C9000331241B5E0F40495
:10243B002546FEE56C90002D1241B5EEF08017E5B8
:10244B006C9000331241B5E0C39546FEE56C9000ED
:10245B002D1241B5EEF0E56C6029E56C90002D1264
:10246B0041B5FEE0FFEE900031E0D39F4013E56CE9
:10247B0090002D1241B5E0900031F0E56C900032E8
:10248B00F0800E90002DE0900031F074009000323F
:10249B00F0786C740126F64003022418900082E059
:1024AB007043E52A45296036E558C39403500A90DA
:1024BB000032E004C3940340028007900032E00432
:1024CB00F558E558D39402400A900032E004D394B7
:1024DB000250028007900032E004F558800790000C
:1024EB0032E004F55875BB180543D2ECE55FD39485
:1024FB0004500302260B75CF01C2A2AE35AF367462
:10250B0088D39F74139E4005A2A5B34014AE35AF7C
:10251B00367488D39F74139E4005A2A4B3400280E7
:10252B0048783512003FAE35AF36EFB4883BEEB48A
:10253B001337A2A5B3500990004FE0D39551500229
:10254B00800405518011A2A5B3500890004FE0659F
:10255B005160028002D207A2A4B35007E551D39475
:10256B0001500280041551C207A2A5B3B35006A2B5
:10257B00A4B3B340028006753600753500E551658E
:10258B0052604EE55175F040A4FFAEF0900322125D
:10259B00001EE030E003D38001C39296E55175F045
:1025AB0040A4FFAEF090032312001EE030E003D3F3
:1025BB008001C39295E55175F040A4FFAEF09003F6
:1025CB002412001EE030E003D38001C392A085519A
:1025DB0052900083E06005A2B2B340028004C29720
:1025EB008002D297A20740057572CD80037572FFEA
:1025FB00E595C395724004C2A18002D2A1022501C8
:10260B00A20EB3500DAE25AF2674E8C39F74039E84
:10261B004002800575FFA0D20EAE25AF26EFD394F6
:10262B0020EE944E500302271F120481C28E758D2B
:10263B0000758B00754C00D28EC2077571007570DA
:10264B00007572CD75510475240075230075540007
:10265B00755A00C287900059E06004D2908002C284
:10266B009090004AE0B40104D2948002C29490008E
:10267B0049E0B40104D2938002C293A209B340048F
:10268B00D2918002C29190006BE060181237F2A2D7
:10269B0000B34008E5B54408F5B58006E5B554F739
:1026AB00F5B58002C20090006EE06018123947A2A7
:1026BB0002B34008E5B54402F5B58006E5B554FD17
:1026CB00F5B58006E5B554FDF5B590000E74FDF03B
:1026DB00A374E8F0E543B40603754300900025E4CA
:1026EB00F0752600752500758D00758B00754C00F7
:1026FB00900024E0C394035008900024E004F08081
:10270B00067403900024F0900024E0B40306E5B5B2
:10271B0054FEF5B5AE27AF28EFD39410EE942740B7
:10272B001CC2CA75CD0075CC00752800752700D268
:10273B00CA754E00752A00752900755500020CCC20
:103AF90000000100013201640196019602000212E0
:103B090002240200020003000340038003C00400F2
:103B19000440048004C005000600060006000600F3
:103B2900060006000600060000FF01310163019549
:103B390001FF01FF0211022302FF02FF02FF033FFF
:103B4900037F03BF03FF043F047F04BF04FF05FF96
:103B590006FF06FF06FF06FF06FF06FF06FF06FF34
:103B69000FAA0FA50F9F0F9A0F940F8D0F870F8024
:103B79000F780F710F680F600F570F4E0F450F3BEE
:103B89000F300F250F1A0F0E0F020EF50EE80EDB80
:103B99000ECC0EBE0EAE0E9F0E8E0E7D0E6C0E5A04
:103BA9000E470E340E200E0C0DF70DE20DCB0DB5A0
:103BB9000D9D0D850D6D0D540D3A0D200D050CE96A
:103BC9000CCE0CB10C940C760C580C3A0C1B0BFB5C
:103BD9000BDB0BBB0B9A0B790B570B350B130AF14C
:103BE9000ACE0AAB0A870A640A400A1C09F809D4F2
:103BF90009B0098C09670943091F08FB08D608B2EF
:103C0900088E086A0846082307FF07DC07B90796E4
:103C190007730751072F070D06EC06CA06AA06897E
:103C290006690649062A060A05EC05CD05B005927E
:103C390005750558053C0520050504EA04CF04B5BA
:103C4900049C04820469045104390422040B03F41A
:103C590003DE03C803B2039D038903750361034DA2
:103C6900033B03280316030402F202E102D102C056
:103C790002B002A002910282027302650257024950
:103C8900023C022F02220216020901FD01F201E69D
:103C990001DB01D001C601BB01B101A7019D01945E
:103CA900018B01820179017001680160015801509D
:103CB9000148014101390132012B0125011E011879
:103CC9000111010B010500FF00FA0FA60FA00F99C2
:103CD9000F920F8B0F840F7C0F740F6B0F620F58AD
:103CE9000F4E0F430F380F2C0F1F0F120F050EF732
:103CF9000EE80ED80EC80EB70EA50E930E800E6CE8
:103D09000E580E420E2C0E150DFD0DE40DCB0DB106
:103D19000D950D790D5D0D3F0D200D010CE10CC0C8
:103D29000C9E0C7C0C590C350C100BEA0BC40B9E29
:103D39000B760B4F0B260AFD0AD40AAA0A800A55EC
:103D49000A2A09FF09D409A8097C0950092508F993
:103D590008CD08A10875084A081E07F307C8079D7A
:103D690007730749072006F706CE06A6067E0657FB
:103D79000630060A05E405BF059B0577055405329B
:103D8900051004EF04CE04AE048F04710453043506
:103D9900041903FD03E203C703AD0394037B036323
:103DA900034B0334031E030802F302DE02CA02B600
:103DB90002A30291027F026D025C024C023C022CBA
:103DC900021D020E020001F201E401D701CA01BE7F
:103DD90001B101A6019A018F0185017A017001667D
:103DE900015D0153014A01410139013101290121D3
:103DF90001190112010B010400FD00F700F000EAAE
:103E090000E400DE00D900D300CE00C900C400BF21
:103E190000BA00B500B100AD00A800A400A0009C44
:103E2900009900950091008E008A00870084008126
:043E3900007E007B8C
:10276C00751A00751900AE19AF1AAC17AD18EDC378
:10277C009FEC9E401674FF12416F75CF01781A744E
:10278C000126F6500418E436F650DB22900786E456
:10279C00F0A3F0751000750F00751300751400C2CE
:1027AC0010D21122C2AF75D900758F0375B7A575FC
:1027BC00B7F190F800E4F0758F0175B7A575B7F116
:1027CC00E50890F800F075B7A575B7F190F801E43D
:1027DC00F075B7A575B7F190079DE090F802F0750C
:1027EC00B7A575B7F19007A1E090F803F075B7A500
:1027FC0075B7F190079EE090F804F075B7A575B722
:10280C00F190079FE090F805F075B7A575B7F190BA
:10281C0007A0E090F806F075B7A575B7F19007A280
:10282C00E090F807F0758F0075D940D2AF22900771
:10283C0088E0B4AB61C2AF75D90075B62275F522CC
:10284C00758F0375B7A575B7F1740090F600F07528
:10285C008F01750A00750900AE09AF0A7413BE002A
:10286C00279F402475B7A575B7F190078912001EF4
:10287C00E0FC90F60012001EECF0780A740126F6CB
:10288C00500418E436F650D0758F0075F51175B6F6
:10289C002075D940D2AF22C2AF75D90075F522751B
:1028AC000A00750900AE09AF0A7413BE00229F40DE
:1028BC001F90F60012001EE493FC90078912001E74
:1028CC00ECF0780A740126F6500418E436F650D56C
:1028DC0075F51175D940D2AF22900788E0B4AA02E1
:1028EC008003022A22C2AF75D90075B62275F52273
:1028FC00758F0375B7A575B7F1740090EE00F07580
:10290C00B7A575B7F1740090F000F075B7A575B761
:10291C00F1740090F200F075B7A575B7F1740090E2
:10292C00F400F0758F01750A00750900AE09AF0A45
:10293C0074FFC39F74019E402475B7A575B7F190C1
:10294C00004E12001EE0FC90EE0012001EECF0781F
:10295C000A740126F6500418E436F650CF750A00B6
:10296C00750900AE09AF0A74FFC39F74019E402421
:10297C0075B7A575B7F190024E12001EE0FC90F0F1
:10298C000012001EECF0780A740126F6500418E4CC
:10299C0036F650CF750A00750900AE09AF0A74FF00
:1029AC00C39F74019E402475B7A575B7F190044E72
:1029BC0012001EE0FC90F20012001EECF0780A747B
:1029CC000126F6500418E436F650CF750A00750946
:1029DC0000AE09AF0A74FFC39F74019E402475B703
:1029EC00A575B7F190064E12001EE0FC90F4001293
:1029FC00001EECF0780A740126F6500418E436F642
:102A0C0050CF758F0075F51175B62075D940D2AFC2
:102A1C00743A90074EF022900788E0B4AA02800323
:102A2C00022B60C2AF75D90075B62275F522758F71
:102A3C000375B7A575B7F1740090E600F075B7A5EE
:102A4C0075B7F1740090E800F075B7A575B7F1741F
:102A5C000090EA00F075B7A575B7F1740090EC0022
:102A6C00F0758F01750A00750900AE09AF0A74FF85
:102A7C00C39F74019E402475B7A575B7F190004EA5
:102A8C0012001EE0FC90E60012001EECF0780A74B6
:102A9C000126F6500418E436F650CF750A00750975
:102AAC0000AE09AF0A74FFC39F74019E402475B732
:102ABC00A575B7F190024E12001EE0FC90E80012D2
:102ACC00001EECF0780A740126F6500418E436F671
:102ADC0050CF750A00750900AE09AF0A74FFC39F89
:102AEC0074019E402475B7A575B7F190044E120081
:102AFC001EE0FC90EA0012001EECF0780A7401262D
:102B0C00F6500418E436F650CF750A00750900AE7D
:102B1C0009AF0A74FFC39F74019E402475B7A57555
:102B2C00B7F190064E12001EE0FC90EC0012001E55
:102B3C00ECF0780A740126F6500418E436F650CFFF
:102B4C00758F0075F51175B62075D940D2AF743AF2
:102B5C0090074EF022900788E0B4AA028003022C62
:102B6C009EC2AF75D90075B62275F522758F0375A7
:102B7C00B7A575B7F1740090DE00F075B7A575B701
:102B8C00F1740090E000F075B7A575B7F174009082
:102B9C00E200F075B7A575B7F1740090E400F0751C
:102BAC008F01750A00750900AE09AF0A74FFC39F47
:102BBC0074019E402475B7A575B7F190004E1200B4
:102BCC001EE0FC90DE0012001EECF0780A74012668
:102BDC00F6500418E436F650CF750A00750900AEAD
:102BEC0009AF0A74FFC39F74019E402475B7A57585
:102BFC00B7F190024E12001EE0FC90E00012001E95
:102C0C00ECF0780A740126F6500418E436F650CF2E
:102C1C00750A00750900AE09AF0A74FFC39F7401F1
:102C2C009E402475B7A575B7F190044E12001EE0B6
:102C3C00FC90E20012001EECF0780A740126F650AB
:102C4C000418E436F650CF750A00750900AE09AFCA
:102C5C000A74FFC39F74019E402475B7A575B7F124
:102C6C0090064E12001EE0FC90E40012001EECF0E8
:102C7C00780A740126F6500418E436F650CF758F96
:102C8C000075F51175B62075D940D2AF743A90071E
:102C9C004EF022900788E0B4AA028003022DDCC219
:102CAC00AF75D90075B62275F522758F0375B7A56A
:102CBC0075B7F1740090D600F075B7A575B7F174BF
:102CCC000090D800F075B7A575B7F1740090DA00D4
:102CDC00F075B7A575B7F1740090DC00F0758F0135
:102CEC00750A00750900AE09AF0A74FFC39F740121
:102CFC009E402475B7A575B7F190004E12001EE0EA
:102D0C00FC90D60012001EECF0780A740126F650E6
:102D1C000418E436F650CF750A00750900AE09AFF9
:102D2C000A74FFC39F74019E402475B7A575B7F153
:102D3C0090024E12001EE0FC90D80012001EECF027
:102D4C00780A740126F6500418E436F650CF750A4A
:102D5C0000750900AE09AF0A74FFC39F74019E4051
:102D6C002475B7A575B7F190044E12001EE0FC90C7
:102D7C00DA0012001EECF0780A740126F6500418E2
:102D8C00E436F650CF750A00750900AE09AF0A7427
:102D9C00FFC39F74019E402475B7A575B7F19006CB
:102DAC004E12001EE0FC90DC0012001EECF0780AC3
:102DBC00740126F6500418E436F650CF758F007562
:102DCC00F51175B62075D940D2AF743A90074EF014
:102DDC0022C2AF75D90075F522750A00750900AECF
:102DEC0009AF0A74FFC39F74019E401F90EE00123E
:102DFC00001EE493FC90004E12001EECF0780A7456
:102E0C000126F6500418E436F650D4750A007509FC
:102E1C0000AE09AF0A74FFC39F74019E401F90F06F
:102E2C000012001EE493FC90024E12001EECF0788F
:102E3C000A740126F6500418E436F650D4750A00CC
:102E4C00750900AE09AF0A74FFC39F74019E401F41
:102E5C0090F20012001EE493FC90044E12001EEC43
:102E6C00F0780A740126F6500418E436F650D4753E
:102E7C000A00750900AE09AF0A74FFC39F74019E66
:102E8C00401F90F40012001EE493FC90064E1200BA
:102E9C001EECF0780A740126F6500418E436F6504D
:102EAC00D475F51175D940D2AF22C2AF75D9007562
:102EBC00F522750A00750900AE09AF0A74FFC39FAD
:102ECC0074019E401F90E60012001EE493FC9000DB
:102EDC004E12001EECF0780A740126F6500418E429
:102EEC0036F650D4750A00750900AE09AF0A74FFA6
:102EFC00C39F74019E401F90E80012001EE493FCD7
:102F0C0090024E12001EECF0780A740126F6500462
:102F1C0018E436F650D4750A00750900AE09AF0AEC
:102F2C0074FFC39F74019E401F90EA0012001EE4C0
:102F3C0093FC90044E12001EECF0780A740126F6F5
:102F4C00500418E436F650D4750A00750900AE0921
:102F5C00AF0A74FFC39F74019E401F90EC001200D7
:102F6C001EE493FC90064E12001EECF0780A7401DD
:102F7C0026F6500418E436F650D475F51175D94080
:102F8C00D2AF22C2AF75D90075F522750A0075094A
:102F9C0000AE09AF0A74FFC39F74019E401F90DE00
:102FAC000012001EE493FC90004E12001EECF07810
:102FBC000A740126F6500418E436F650D4750A004B
:102FCC00750900AE09AF0A74FFC39F74019E401FC0
:102FDC0090E00012001EE493FC90024E12001EECD6
:102FEC00F0780A740126F6500418E436F650D475BD
:102FFC000A00750900AE09AF0A74FFC39F74019EE5
:10300C00401F90E20012001EE493FC90044E12004C
:10301C001EECF0780A740126F6500418E436F650CB
:10302C00D4750A00750900AE09AF0A74FFC39F740A
:10303C00019E401F90E40012001EE493FC90064E8B
:10304C0012001EECF0780A740126F6500418E436CF
:10305C00F650D475F51175D940D2AF22C2AF75D9DF
:10306C000075F522750A00750900AE09AF0A74FFE8
:10307C00C39F74019E401F90D60012001EE493FC67
:10308C0090004E12001EECF0780A740126F65004E3
:10309C0018E436F650D4750A00750900AE09AF0A6B
:1030AC0074FFC39F74019E401F90D80012001EE451
:1030BC0093FC90024E12001EECF0780A740126F676
:1030CC00500418E436F650D4750A00750900AE09A0
:1030DC00AF0A74FFC39F74019E401F90DA00120068
:1030EC001EE493FC90044E12001EECF0780A74015E
:1030FC0026F6500418E436F650D4750A007509000B
:10310C00AE09AF0A74FFC39F74019E401F90DC0090
:10311C0012001EE493FC90064E12001EECF0780A8E
:10312C00740126F6500418E436F650D475F5117572
:10313C00D940D2AF22E51464046006E59964FF60BF
:10314C00028031A2104004D2108027E5146008746C
:10315C00E62514900023F0E513600874F025139015
:10316C000023F0E514B4010280FE75140075130001
:10317C00C2108002C210E514903A9CF8282873758E
:10318C001400E599B4FF03751301E599B4FE0375BA
:10319C001302E599B4FD03751303E599B4FC0375AB
:1031AC001304E599B4FA03751305E599B4FB067598
:1031BC001401120481E599B4F90675140412048102
:1031CC00E599D394E54007E599C394F04002801645
:1031DC008599157514027E017F00E515C394E612DE
:1031EC00419D8E0D8F0E900786E4F0A3F0E599D3E8
:1031FC0094C44007E599C394E6400280288599154C
:10320C0075140374E5C39515F50E750D00AE0DAF71
:10321C000E903AF912002EE493F8740193900786FD
:10322C00C8F0A3C8F0D2990236B0900786E0FEA38E
:10323C00E0FFEFC39400EE94054009EFD394FFEE4A
:10324C0094064013900786E0FEA3E0FF90004E1218
:10325C00001EE599F0800385996D90078612000E8B
:10326C00900786E0FEA3E0FFEFB40106EEB4070280
:10327C0080030234C090074EE0B43C028003023459
:10328C00C0A20AB35005A20BB340030233B3C29CD5
:10329C0090007AE090078CF0900057E090078DF04A
:1032AC00900062E090078EF0900063E090078FF042
:1032BC00900074E0900790F090007CE0900791F003
:1032CC0090007DE0900792F0900080E0900793F0E2
:1032DC00900081E0900794F090013AE0900795F00F
:1032EC0090013BE0900796F090013CE0900797F03E
:1032FC00900090E0900798F0900091E0900799F082
:10330C00900092E090079AF0900093E090079BF069
:10331C00900094E090079CF0900095E090079DF051
:10332C00900096E090079EF0900097E090079FF039
:10333C00900099E09007A0F090009AE09007A1F01F
:10334C0090009BE09007A2F090009CE09007A3F007
:10335C007400900082F01200C974AB900788F012D0
:0A336C00283A74AA900788F0E5588B
:063A9C0002318B023236FC
:10337600903ABDF828287380121228E5800D122A8B
:0B338600238008122B618003122C9F93
:0F3ABD0002337D02337F02338402338902338E5A
:10339100900788E4F090013AE0700C90013BE070F6
:1033A1000690013CE060028004C20A8002D20A0257
:1033B10034B5C29C900078E0900789F090005EE0FF
:1033C10090078AF090005FE090078BF090007AE020
:1033D10090078CF0900057E090078DF0900062E02C
:1033E10090078EF0900063E090078FF0900074E0FA
:1033F100900790F090007CE0900791F090007DE0C4
:10340100900792F0900080E0900793F0900081E0A7
:10341100900794F090013AE0900795F090013BE01D
:10342100900796F090013CE0900797F0900090E0B3
:10343100900798F0900091E0900799F0900092E049
:1034410090079AF0900093E090079BF0900094E031
:1034510090079CF0900095E090079DF0900096E019
:1034610090079EF0900097E090079FF0900099E000
:103471009007A0F090009AE09007A1F090009BE0E7
:103481009007A2F090009CE09007A3F074009000D8
:1034910082F074AB900788F012283A74AA900788DA
:1034A100F01228E5122A23122B61122C9FD29C754F
:1034B10099FB80FED29C7514007513007599FB026F
:1034C10036B0900786E0FEA3E0FFEF4E70068599C7
:1034D10010750F00900786E0FEA3E0FF74016F4EA8
:1034E100701BAC0FAD10AA0DAB0EED2BFBEC3AFA35
:1034F1008A068B0790004E12001EE599F090078610
:1035010012000E900786E0FEA3E0FF74026F4E707A
:103511000C1200C98515997514007513000236B097
:10352100900786E0FEA3E0FF90004E12001EE59991
:10353100F090078612000E900786E0FEA3E0FFAC34
:103541000DAD0E8F028E038C068D07903B3112005C
:103551002EE493F9740193FEEAD39EEB9940098519
:1035610015997514007513000236B0900786E0FEB8
:10357100A3E0FF90004E12001EE599F0900786121D
:10358100000E900786E0FEA3E0FFEFB40006EEB464
:10359100010280030236B090001CE0D394C7400BB7
:1035A10090001CE0C394C8F516801A90001CE0D36B
:1035B1009463400B90001CE0C39464F51680069060
:1035C100001CE0F516E51675F002A4FFAEF08F6C55
:1035D100EF90004E1241B5EFFCE0FDEC900051126E
:1035E10041B5EDFCE0FDEC2DB5160280030236A2DB
:1035F1000FEF90004E1241B5E56CFFE0FCEF90003B
:10360100521241B5ECFFE0FCEFC39CB516028003FA
:103611000236A2E56C9000501241B5E56CFFE0FC6A
:10362100EF9000531241B5ECFFE0FCEF2CB51671A1
:10363100E56C9000541241B5E0C3951690079DF0DA
:10364100E56C9000551241B5E0C3951690079EF0C8
:10365100E56C9000581241B5E0C3951690079FF0B4
:10366100E56C9000591241B5E0C395169007A0F0A2
:10367100E56C90005A1241B5E0C395169007A1F090
:10368100E56C90005B1241B5E0C395169007A2F07E
:103691001227B07599F975186475170012276C8097
:0F36A100FE7599FF75186475170012276C80FE6F
:093AA2000234C302352102356C27
:1036B00022E513903AABF82828730237F190078679
:1036C000E0FEA3E0FF90001212001EE0F5999007C3
:1036D0008612000E900786E0FEA3E0FF74116F4E85
:1036E00070037513000237F18563990237F1900773
:1036F00086E0FEA3E0FF90004E12001EE0F599EF79
:10370000B40107EEB4070375130090078612000E8C
:073710000237F1900787E08A
:0F3AAB000236BA0236BD0236E80236EE02371393
:10371700903ACCF82828738524990237E6852A99A8
:103727000237E68544990237E68547990237E685E9
:1037370051990237E68561990237E685569902372E
:10374700E68558990237E6756F00900069E07006C4
:10375700900068E060028016A2A44006E56F44046A
:10376700F56FA2A54006E56F4402F56F801A900039
:103777004AE0B40106E56F4410F56F900049E0B4E4
:103787000106E56F4420F56FA207B34006E56F44D5
:1037970001F56FA209B34006E56F4408F56F856F21
:1037A70099803CA211B340077599FAC2118017A2FC
:1037B7000CB3400575990F800B900023E0F59990A5
:1037C7000023E4F0C20C80178542998012854B993B
:0F37D700800D85469980087599FC800375130055
:103ACC0002371E02372402372A02373002373602F9
:103ADC00373C02374202374802374E0237AA0237C8
:0D3AEC00CF0237D40237D90237DE0237E3AC
:0B37E60090078612000E8003120048BE
:033ABA000237EEE2
:1037F1002290006BE0B4010385241190006BE0B4CA
:103801000203852A1190006BE0B4030385441190F3
:10381100006BE0B4040385471190006BE0B405032D
:1038210085511190006BE0B4060385561190006B31
:10383100E0B4070385581190006CE0FE90006DE044
:10384100C39E50030238C890006BE0D39404402C0F
:1038510090006CE0D39511500990006DE0C3951173
:1038610050028002D20090006CE0D3951150099073
:10387100006DE0C395115002C200804990006BE0D9
:10388100B4041890006DE0C395115002D20090006D
:103891006CE0D395114002C200802A90006CE0C315
:1038A1009511500990006DE0D3951150028002D21C
:1038B1000090006CE0D39511500990006DE0C39524
:1038C100115002C200807E90006BE0D39404402C22
:1038D10090006CE0C39511400990006DE0D3951103
:1038E10040028002C20090006CE0C3951140099033
:1038F100006DE0D395114002D200804990006BE049
:10390100B4041890006CE0C395115002C2009000FD
:103911006DE0D395114002D200802A90006CE0C383
:103921009511400990006DE0D395114002D20090AD
:10393100006CE0D39511400990006DE0C3951140F2
:10394100028002C2002290006EE0B40103852411BE
:1039510090006EE0B40203852A1190006EE0B4037A
:103961000385441190006EE0B40403854711900073
:103971006EE0B4050385511190006EE0B406038535
:10398100561190006EE0B4070385581190006FE066
:10399100FE900070E0C39E5003023A1D90006EE05D
:1039A100D39404402C90006FE0D3951150099000FE
:1039B10070E0C3951150028002D20290006FE0D3F3
:1039C10095115009900070E0C395115002C2028018
:1039D1004990006EE0B40418900070E0C395115056
:1039E10002D20290006FE0D395114002C202802AF8
:1039F10090006FE0C395115009900070E0D39511CC
:103A010050028002D20290006FE0D39511500990CC
:103A11000070E0C395115002C202807E90006EE0FA
:103A2100D39404402C90006FE0C39511400990009D
:103A310070E0D3951140028002C20290006FE0C392
:103A410095114009900070E0D395114002D2028097
:103A51004990006EE0B4041890006FE0C3951150D6
:103A610002C202900070E0D395114002D202802A76
:103A710090006FE0C395114009900070E0D395115B
:103A81004002D20290006FE0D3951140099000707E
:0B3A9100E0C3951140028002C2022237
:0941B5002582F5825002058322E7
:10002E00EF2F500205832582F582E5833E2EF58360
:01003E00229F
:08000300C3EF9DFFEE9CFE22FD
:08003F000806B60002180622B3
:0D000E00A3E004F070061241ABE004F02204
:0841C7000816B6FF02181622CB
:0E418F00048007C3CE13CECF13CFD5E0F622A7
:10403D00BC000FBE0008ED8FF084FFADF022E4FE52
:10404D00FF22BE000DEF60FE54F0606F20E703020B
:10405D0040F3EAC0E0EBC0E078017A0075F001EEC4
:10406D0020E710EF25E0FFEE33FE0AC5F023C5F083
:10407D0030E7F0EA5407F9096A7A007B006001081D
:10408D00C3EC9E40167004ED9F4010ED9FFDEC9E1D
:10409D00FCE5F0CA4ACA03F5F08005E5F003F5F03A
:1040AD00C3EE13FEEF13FFD9D77908CACBCAD8D008
:1040BD00EAFEEBFFD0E0FBD0E0FA22EC8FF084FCBF
:1040CD00ED54F045F0C48FF084FEEDC454F045F08E
:1040DD00C48FF084FDEEC4FE54F02DFFEE540F3C62
:1040ED00FEADF07C0022790078008FF0EC7E082088
:1040FD00E70DC3CD33CD33C933C9C833C8DEF08422
:10410D0049F9E5F08FF0BE00E6FD7C00E9FFE8FE21
:01411D00227F
:0E419D00F88FF0A4FFE5F0CE88F0A42EFE22ED
:10416F00600D782B024179007830D8FED5E0F82227
:10417F00EEC0E07E0012403DEFFDEEFCD0E0FE22EF
:03000B0002411E91
:03001B0002413966
:03002B000241543B
:030000000241BEFC
:0941BE0075817375D0000207FF42
:0B001E00E5822FF582E5833EF583228A
:0A41AB000582D582021583158222D9
:10411E00C0E0C0F0C083C082C0D075D0001207F4DA
:10412E00D0D0D082D083D0F0D0E032C0E0C0F0C08A
:10413E0083C082C0D075D0001207F7D0D0D082D005
:10414E0083D0F0D0E032C0E0C0F0C083C082C0D0D7
:10415E0075D0001207FAD0D0D082D083D0F0D0E044
:01416E00321E
:00000001FF
